:1000000023C03BC0CCC239C038C037C0DEC135C008
:1000100034C033C032C031C030C02FC02EC02DC05C
:100020002CC02BC02AC044544D46204465636F64E5
:100030006572206279207777772E696E66696469C8
:10004000676D2E6E6574000011241FBECFEDCDBF0D
:1000500010E0A0E6B0E0EAE0F6E003C0C895319613
:100060000D92A036B107D1F710E0A0E6B0E001C0D4
:100070001D92AA37B107E1F79DC0C2CF982F869590
:100080008EBBE09A90FF05C08DB399278F7090705A
:1000900008958DB382958F70992708950895CF9311
:1000A000DF93CDB7DEB722970FB6F894DEBF0FBE51
:1000B000CDBF9FEF97BB813011F4959A01C0959801
:1000C00068BB19821A8289819A81C29730F489812A
:1000D0009A81019689839A83F6CF969A19821A8219
:1000E00089819A81C29730F489819A8101968983A6
:1000F0009A83F6CF969819821A8289819A81883CD0
:10010000910530F489819A81019689839A83F5CF8C
:1001100017BA22960FB6F894DEBF0FBECDBFDF919F
:10012000CF9108955D9BFECF8CB908950F931F93D7
:10013000CF93DF93D92FC82F00E060E8802FAFDF87
:10014000FD2FEC2FC895802D8823B9F0FD2FEC2FC3
:10015000C895102D1CB9003119F460EC80E09FDFC8
:10016000612F81E09CDF21960F5F5D9BFECFFD2F0D
:10017000EC2FC895802D882349F7DF91CF911F91EF
:100180000F9108958F3019F480E290E008958A303D
:1001900019F480E390E008958B3019F48AE290E03E
:1001A00008958C3019F483E290E0089580639927D4
:1001B00008950895CFEDD0E0DEBFCDBFF89417BA13
:1001C00080E781BBC49886E189B988E08AB983E079
:1001D00083BF82E089BF90E89BBF8CE285BF9ABF56
:1001E000109264008091640049DF8F3039F0809173
:1001F00064008F5F809364008F3FA1F7809164005B
:100200008093780083E18093620081E080937300A3
:10021000682F80E044DF62E080E041DF68E380E057
:100220003EDF6CE080E03BDF66E080E038DF8DE0C1
:1002300079DF8AE077DF86E290E078DF8DE072DFB9
:100240008AE070DF109279008091790090916400CB
:10025000890F8F5F13DF96DF65DF809179008F5FF5
:10026000809379008F3F81F78DE05CDF8AE05ADF71
:1002700078948895FECF1F93CF93C82F162F8A307E
:1002800020F460E281E00BDF04C061E381E007DF7E
:10029000CA50C0636C2F81E002DF6DE281E0FFDEB7
:1002A000C1E0809178008C0F811B8E50E7DE6ADF01
:1002B000682F81E0F4DECF5FCE3098F3CF911F91AD
:1002C000089561E381E0EBDE69E381E0E8DE6DE261
:1002D00081E0E5DE1092790080917200882391F030
:1002E00080917900E82FFF27EB59FF4F608181E073
:1002F000D6DE809179008F5F8093790090917200B3
:10030000891770F30895CF93C82F609173006130FF
:10031000A1F4809172008D3080F4109273001092DD
:10032000600083E18093620080E0B9DE60E082E1FA
:10033000A2DF60EC80E0B3DEC4DF809172008D301C
:10034000A8F161E080E0ABDE61E381E0A8DE68E374
:1003500081E0A5DE6DE281E0A2DE10927200809164
:100360007200E82FFF27EB59FF4F608181E097DE95
:10037000809172008F5F809372008E3080F360EC0A
:1003800080E08DDE61E381E08ADE69E381E087DE83
:100390006DE281E084DE10927200809164008093AF
:1003A00078001092600083E1809362006C2F81E0FE
:1003B00076DE80917200E82FFF27EB59FF4FC08354
:1003C0008F5F80937200CF9108951F920F920FB6A6
:1003D0000F9211241F932F933F934F935F936F932B
:1003E0007F938F939F93AF93BF93CF93EF93FF939D
:1003F000809B0EC086E180937400809176008631E8
:1004000020F48F5F8093760042C0109261003FC05D
:100410001092760080917400882321F0815080939F
:10042000740035C0C0916100CC2389F580916200D1
:10043000833168F511E010937300810F809362009F
:10044000612F8C2F2CDE809160008D509091620086
:10045000682F892F81500FDF60EC8C2F20DE909168
:100460006200933131F0809160008A51682F892FAA
:1004700002DF809160008D50809360008091620067
:10048000833119F41EDFC093730010936100829BC7
:100490000EC086E18093750080917700863120F44C
:1004A0008F5F8093770036C01092630033C0109244
:1004B000770080917500882321F08150809375002A
:1004C00029C0C0916300CC2329F58091620083305C
:1004D00008F111E010937300815080936200612F46
:1004E0008C2FDDDD80916000835F90916200682F2A
:1004F000892F8150C0DE60EC8C2FD1DD60916000CF
:1005000080916200B8DE80916000835F809360001C
:1005100010936300FF91EF91CF91BF91AF919F91A5
:100520008F917F916F915F914F913F912F911F918B
:100530000F900FBE0F901F901895F894E199FECF81
:1005400086958EBB6DBBE29AE19A78940895CF931D
:10055000C82F8091640080FF16C081508FDD682F06
:100560006295607F6C2B80916400E7DF809164006E
:100570008F5F809364008F5F81DD682F606F809153
:100580006400DBDF0AC0C295C07FCF606C2FD5DF6F
:10059000809164008F5F80936400CF9108951F92D3
:1005A0000F920FB60F9211240F931F932F933F9327
:1005B0004F935F936F937F938F939F93AF93BF936B
:1005C000EF93FF93F89417BA949A000016B3949897
:1005D0001F70812FD7DD082F96DE812FB8DF802F87
:1005E000A1DD7894FF91EF91BF91AF919F918F9191
:1005F0007F916F915F914F913F912F911F910F913B
:0A0600000F900FBE0F901F90189589
:00000001FF
